******************************************************************************
               TMS320C6x Linker PC v7.4.8                      
******************************************************************************
>> Linked Mon Aug 24 09:12:46 2015

OUTPUT FILE NAME:   <AM57xx_DSP2DEMO.out>
ENTRY POINT SYMBOL: "_c_int00"  address: 00800000


MEMORY CONFIGURATION

         name            origin    length      used     unused   attr    fill
----------------------  --------  ---------  --------  --------  ----  --------
  entry_point           00800000   00000080  00000080  00000000  RWIX
  DSPL2RAM              00800080   0003ff00  00000000  0003ff00  RWIX
  DSPL1PRAM             00e00000   00008000  00000000  00008000  RWIX
  DSPL1DRAM             00f00000   00008000  00000000  00008000  RWIX
  DSP_PROG              9f000080   00700000  00003220  006fcde0  RWIX


SEGMENT ALLOCATION MAP

run origin  load origin   length   init length attrs members
----------  ----------- ---------- ----------- ----- -------
00800000    00800000    00000080   00000080    r-x
  00800000    00800000    00000080   00000080    r-x .text:_c_int00
9f000080    9f000080    00000240   00000000    rw-
  9f000080    9f000080    00000240   00000000    rw- .far
9f0002c0    9f0002c0    0000000c   0000000c    rw-
  9f0002c0    9f0002c0    0000000c   0000000c    rw- .fardata
9f0002cc    9f0002cc    00000034   00000034    r--
  9f0002cc    9f0002cc    00000034   00000034    r-- .cinit
9f000400    9f000400    00002ba0   00002ba0    r-x
  9f000400    9f000400    00002ba0   00002ba0    r-x .text
9f002fa0    9f002fa0    00000400   00000000    rw-
  9f002fa0    9f002fa0    00000400   00000000    rw- .stack


SECTION ALLOCATION MAP

 output                                  attributes/
section   page    origin      length       input sections
--------  ----  ----------  ----------   ----------------
.init_array 
*          0    9f000080    00000000     UNINITIALIZED

.text:_c_int00 
*          0    00800000    00000080     
                  00800000    00000080     rts6600_elf.lib : boot.obj (.text:_c_int00)

.far       0    9f000080    00000240     UNINITIALIZED
                  9f000080    00000240     interrupt.obj (.far)

.fardata   0    9f0002c0    0000000c     
                  9f0002c0    0000000c     rts6600_elf.lib : exit.obj (.fardata)

.cinit     0    9f0002cc    00000034     
                  9f0002cc    0000000d     (.cinit..fardata.load) [load image, compression = rle]
                  9f0002d9    00000003     --HOLE-- [fill = 0]
                  9f0002dc    0000000c     (__TI_handler_table)
                  9f0002e8    00000008     (.cinit..far.load) [load image, compression = zero_init]
                  9f0002f0    00000010     (__TI_cinit_table)

.text      0    9f000400    00002ba0     
                  9f000400    00001aa0     interrupt.obj (.text:retain)
                  9f001ea0    000005e0     interrupt.obj (.text)
                  9f002480    000001a0     main.obj (.text)
                  9f002620    00000180     rts6600_elf.lib : copy_decompress_rle.obj (.text:__TI_decompress_rle_core)
                  9f0027a0    00000060                     : cpp_init.obj (.text:__TI_cpp_init)
                  9f002800    00000200     intvecs.obj (.text)
                  9f002a00    00000100     rts6600_elf.lib : autoinit.obj (.text:_auto_init_elf)
                  9f002b00    00000100                     : cpy_tbl.obj (.text:copy_in)
                  9f002c00    000000e0                     : copy_zero_init.obj (.text:decompress:ZI:__TI_zero_init)
                  9f002ce0    000000c0                     : exit.obj (.text:exit)
                  9f002da0    000000c0                     : tls.obj (.text:tls:init:__TI_tls_init)
                  9f002e60    000000a0                     : memcpy64.obj (.text:memcpy)
                  9f002f00    00000040                     : args_main.obj (.text:_args_main)
                  9f002f40    00000020                     : exit.obj (.text:abort)
                  9f002f60    00000020                     : copy_decompress_none.obj (.text:decompress:none:__TI_decompress_none)
                  9f002f80    00000020                     : copy_decompress_rle.obj (.text:decompress:rle24:__TI_decompress_rle24)

.stack     0    9f002fa0    00000400     UNINITIALIZED
                  9f002fa0    00000008     rts6600_elf.lib : boot.obj (.stack)
                  9f002fa8    000003f8     --HOLE--


LINKER GENERATED COPY TABLES

__TI_cinit_table @ 9f0002f0 records: 2, size/record: 8, table size: 16
	.fardata: load addr=9f0002cc, load size=0000000d bytes, run addr=9f0002c0, run size=0000000c bytes, compression=rle
	.far: load addr=9f0002e8, load size=00000008 bytes, run addr=9f000080, run size=00000240 bytes, compression=zero_init


LINKER GENERATED HANDLER TABLE

__TI_handler_table @ 9f0002dc records: 3, size/record: 4, table size: 12
	index: 0, handler: __TI_zero_init
	index: 1, handler: __TI_decompress_rle24
	index: 2, handler: __TI_decompress_none


GLOBAL SYMBOLS: SORTED ALPHABETICALLY BY Name 

address    name
--------   ----
9f002f40   C$$EXIT
9f0022f8   ExcCombineAdd
9f002340   ExcCombineRemove
9f0022d8   ExcGlobalEnable
9f001ea0   IntDSPINTCInit
9f002250   IntDisable
9f002220   IntEnable
9f002018   IntEventClear
9f002154   IntEventCombineAdd
9f002050   IntEventCombineInit
9f0021f8   IntEventCombineRegister
9f0021a8   IntEventCombineRemove
9f001f5c   IntEventMap
9f001fe4   IntEventSet
9f0022ac   IntGlobalDisable
9f002298   IntGlobalEnable
9f0022c0   IntGlobalRestore
9f001f10   IntRegister
9f002284   IntReset
9f001f34   IntUnRegister
9f0002f0   __TI_CINIT_Base
9f000300   __TI_CINIT_Limit
9f0002dc   __TI_Handler_Table_Base
9f0002e8   __TI_Handler_Table_Limit
UNDEFED    __TI_INITARRAY_Base
UNDEFED    __TI_INITARRAY_Limit
9f0033a0   __TI_STACK_END
00000400   __TI_STACK_SIZE
00000000   __TI_STATIC_BASE
UNDEFED    __TI_TLS_INIT_Base
UNDEFED    __TI_TLS_INIT_Limit
00000001   __TI_args_main
9f0027a0   __TI_cpp_init
9f002f60   __TI_decompress_none
9f002f80   __TI_decompress_rle24
9f0002c8   __TI_enable_exit_profile_output
ffffffff   __TI_pprof_out_hndl
ffffffff   __TI_prof_data_size
ffffffff   __TI_prof_data_start
9f002da0   __TI_tls_init
9f002c00   __TI_zero_init
ffffffff   __binit__
ffffffff   __c_args__
9f002f00   _args_main
9f002a00   _auto_init_elf
9f0013f8   _c674x_mask_int10_isr
9f0015c0   _c674x_mask_int11_isr
9f001784   _c674x_mask_int12_isr
9f001948   _c674x_mask_int13_isr
9f001b10   _c674x_mask_int14_isr
9f001cd8   _c674x_mask_int15_isr
9f000950   _c674x_mask_int4_isr
9f000b18   _c674x_mask_int5_isr
9f000ce0   _c674x_mask_int6_isr
9f000ea4   _c674x_mask_int7_isr
9f001068   _c674x_mask_int8_isr
9f001230   _c674x_mask_int9_isr
9f000400   _c674x_nmi_isr
9f0005c4   _c674x_rsvd_int2_isr
9f000788   _c674x_rsvd_int3_isr
00800000   _c_int00
9f0002c0   _cleanup_ptr
9f0002c4   _dtors_ptr
9f002800   _intcVectorTable
9f002fa0   _stack
9f002f40   abort
ffffffff   binit
9f002b00   copy_in
9f002ce0   exit
9f0025b8   init_irq_crossbar
9f0025e8   main
9f002e60   memcpy
9f0024f8   sendmsg_dsp1
9f0024b8   sendmsg_dsp2
9f002480   sendmsg_mpu


GLOBAL SYMBOLS: SORTED BY Symbol Address 

address    name
--------   ----
00000000   __TI_STATIC_BASE
00000001   __TI_args_main
00000400   __TI_STACK_SIZE
00800000   _c_int00
9f0002c0   _cleanup_ptr
9f0002c4   _dtors_ptr
9f0002c8   __TI_enable_exit_profile_output
9f0002dc   __TI_Handler_Table_Base
9f0002e8   __TI_Handler_Table_Limit
9f0002f0   __TI_CINIT_Base
9f000300   __TI_CINIT_Limit
9f000400   _c674x_nmi_isr
9f0005c4   _c674x_rsvd_int2_isr
9f000788   _c674x_rsvd_int3_isr
9f000950   _c674x_mask_int4_isr
9f000b18   _c674x_mask_int5_isr
9f000ce0   _c674x_mask_int6_isr
9f000ea4   _c674x_mask_int7_isr
9f001068   _c674x_mask_int8_isr
9f001230   _c674x_mask_int9_isr
9f0013f8   _c674x_mask_int10_isr
9f0015c0   _c674x_mask_int11_isr
9f001784   _c674x_mask_int12_isr
9f001948   _c674x_mask_int13_isr
9f001b10   _c674x_mask_int14_isr
9f001cd8   _c674x_mask_int15_isr
9f001ea0   IntDSPINTCInit
9f001f10   IntRegister
9f001f34   IntUnRegister
9f001f5c   IntEventMap
9f001fe4   IntEventSet
9f002018   IntEventClear
9f002050   IntEventCombineInit
9f002154   IntEventCombineAdd
9f0021a8   IntEventCombineRemove
9f0021f8   IntEventCombineRegister
9f002220   IntEnable
9f002250   IntDisable
9f002284   IntReset
9f002298   IntGlobalEnable
9f0022ac   IntGlobalDisable
9f0022c0   IntGlobalRestore
9f0022d8   ExcGlobalEnable
9f0022f8   ExcCombineAdd
9f002340   ExcCombineRemove
9f002480   sendmsg_mpu
9f0024b8   sendmsg_dsp2
9f0024f8   sendmsg_dsp1
9f0025b8   init_irq_crossbar
9f0025e8   main
9f0027a0   __TI_cpp_init
9f002800   _intcVectorTable
9f002a00   _auto_init_elf
9f002b00   copy_in
9f002c00   __TI_zero_init
9f002ce0   exit
9f002da0   __TI_tls_init
9f002e60   memcpy
9f002f00   _args_main
9f002f40   C$$EXIT
9f002f40   abort
9f002f60   __TI_decompress_none
9f002f80   __TI_decompress_rle24
9f002fa0   _stack
9f0033a0   __TI_STACK_END
ffffffff   __TI_pprof_out_hndl
ffffffff   __TI_prof_data_size
ffffffff   __TI_prof_data_start
ffffffff   __binit__
ffffffff   __c_args__
ffffffff   binit
UNDEFED    __TI_INITARRAY_Base
UNDEFED    __TI_INITARRAY_Limit
UNDEFED    __TI_TLS_INIT_Base
UNDEFED    __TI_TLS_INIT_Limit

[75 symbols]
